:04000000C8EF00F055
:0800080000C504F501C505F572
:1000100002C506F5076A03C508F50001F5C409F530
:10002000F6C40AF5F7C40BF5F8C40CF5A1AE1CEF45
:1000300000F0B1BE2EEF00F009C5F5F40AC5F6F4E4
:100040000BC5F7F40CC5F8F404C500F505C501F5BA
:1000500006C502F5078E08C503F511000001C0862C
:1000600003011AA901D0196B070E186F1C511DC38B
:1000700026F5256E2650205C07E303E11F50255C22
:1000800003E21B2AD8B41C2A26C520F525C51FF576
:10009000C096B19E00011CEF00F0C8800301216BE7
:1000A000070E1E6F1F6B206BC882C894C084C89651
:1000B0000001E5EF00F0050EEA6E210EE96EEF504B
:1000C0000EE0140E016E006A002EFED7012EFBD743
:1000D000BF0E006E002EFED700D0EF2EF2D712001A
:1000E000010E245E0CE3050EEA6E240EE96EEF505D
:1000F00006E0040E006E002EFED7EF2EFAD7120097
:10010000C094310E246EECDF1CC523F51BC522F50F
:10011000216A21500F0813E3000B006E2350800B5F
:10012000036E0050031002E0C08401D0C094310E71
:10013000246ED6DFD89022362336212AEAD7C0840F
:10014000310E246ECDDFC094310E246EC9DF1EC582
:1001500023F51DC522F5216A21500F0813E3000B7A
:10016000006E2350800B036E0050031002E0C08429
:1001700001D0C094310E246EB3DFD89022362336DE
:10018000212AEAD7C084310E246EAADF1CEF01F0C9
:10019000F86AD69A078EB06BAF6BB36B080EB16F6F
:1001A000600EAD6F1C6A1B6A206A1F6A0401006B37
:1001B000086B106B206B0001716B726B736B706B53
:1001C000756B766B776B746B68D7B06BAF6BB36B1B
:1001D000030EB16F600EAD6F0A0E216E6CDFB06B57
:1001E000AF6BB36B050EB16F600EAD6F0A0E216E73
:1001F00062DFB06BAF6BB36B080EB16F600EAD6FAB
:1002000003011D6B1C6B00001C511DC303F5800E08
:100210001A6F440E1B6F1AA901D0196B070E186FC5
:10022000A18EC00ED612D0B210D0A19E1C511DC3FB
:100230001EF51D6E000164D703011D6B1C6B0000D1
:0E0240001C6A1B6A206A1F6AA18EEDD703009C
:020000040030CA
:0A0000008CFF36DF9FFFFFFFFFFFBC
:00000001FF
